:1000000010C02AC029C028C027C026C025C024C0CF
:1000100023C022C021C020C01FC03BC01DC01CC0C7
:100020001BC011241FBECFE5D1E0DEBFCDBF10E065
:10003000A0E6B0E0E2E7F1E002C005900D92AE3636
:10004000B107D9F710E0AEE6B0E001C01D92A937C4
:10005000B107E1F75FD08BC0D3CF20E030E040E0C4
:1000600050E0A0EDB7E007C0FD013197F1F72F5F39
:100070003F4F4F4F5F4F2617370748075907A0F3E9
:10008000089598E19DB990E49EB98FB9769BFECF13
:1000900008951F920F920FB60F9211242F938F93F2
:1000A0009F9384B195B19093720080937100809179
:1000B0007100909172008F5F934010F016BE18C0CF
:1000C0008091710090917200499730F486B78F3F0C
:1000D00079F086B78F5F0BC08091710090917200AC
:1000E0004F9730F086B7882319F086B7815086BFC6
:1000F00086B78CBF9F918F912F910F900FBE0F905D
:100100001F9018958CE081B980E887B913B88CEE00
:1001100086B90895F89480EF88BB8BBB8ABB87BBF8
:1001200080E886BD16BC88E18DB9D59A8AB38F7AEE
:100130008ABB80E690E09093760080937500789477
:100140008CE081B980E887B913B88CEE86B983EA70
:1001500080BF82E083BF8AEF86BF8CBFBA9A80EFF0
:100160008ABB8BBB8091710090917200FBCFF89499
:02017000FFCFBF
:0E01720000000002000000004100000000003C
:00000001FF
